:100000000C9484000C94A3000C94A3000C94A30003
:100010000C94A3000C94A3000C949A010C94A300DC
:100020000C94A3000C94A3000C94A3000C94A300C4
:100030000C94A3000C94A3000C94A3000C94A300B4
:100040000C94A3000C94A3000C94A3000C94A300A4
:100050000C9461090C94A3000C94A3000C94A300CD
:100060000C94A3000C94ED100C94B4060C94A30013
:100070000C94A3000C94A3000C94A3000C94A30074
:100080000C94A3000C94A3000C94A3000C94A30064
:100090000C9444120C9470060C94A3000C94A300CE
:1000A0000C94A3000C94A3000C9421010C94A300C5
:1000B0000C94A3000C94A3000C94A3000C94A30034
:1000C0000C94A3000C94A3000C94A300494E464941
:1000D0004E4954594E414ECDCCCC3D0AD7233C1706
:1000E000B7D13877CC2B329595E6241FB14F0A0053
:1000F0000020410000C84200401C4620BCBE4CCA43
:100100001B0E5AAEC59D740011241FBECFEFD1E265
:10011000DEBFCDBF1DE0A0E0B2E0EAEAFCE400E013
:100120000BBF02C007900D92A431B107D9F710E1BF
:10013000A4E1BDE001C01D92AE3AB107E1F70E9413
:10014000801C0C9453260C9400008A3010F4809389
:100150003C0E08951092380E1092390E10923A0EFD
:1001600010923B0E08951092380E1092390E109294
:100170003A0E10923B0E10923C0E82E080933D0EA0
:100180004FEF40937A0E30E130937B0E21E02093C5
:100190007C0E88E998E090937E0E80937D0E1092FD
:1001A0007F0E4093800E3093810E2093820E9093A9
:1001B000840E8093830E3093850E20933E0E109212
:1001C0003F0E1092890E80E090E0FC01EE0FFF1FC1
:1001D000E05CF14F11821082019688309105A9F7F9
:1001E00080E090E0FC01E85CF14F808F0196883060
:1001F0009105C1F780E090E024E6FC01E85CF14F56
:1002000020A3019688309105C1F78FEF9FE390936B
:10021000710E8093700E9093730E8093720E88E02F
:100220008093740E8FEF9FE19093760E8093750EFE
:100230008CE291E09093780E8093770E1092790E75
:1002400008951F920F920FB60F920BB60F921124C2
:100250002F933F934F935F936F937F938F939F93CE
:10026000AF93BF93EF93FF931092A5001092A40059
:100270002091220230912302E0913D0E80918B0D5E
:10028000F0E044E0EE0FFF1F4A95E1F7E80FF11DA3
:10029000EC5DFD4F8081280F311D3093A900209324
:1002A000A8008091180D863034F08FEF90E0909385
:1002B000A9008093A800A8950E9493100E94FB03B8
:1002C000E0913C0E80918B0DF0E034E0EE0FFF1FCB
:1002D0003A95E1F7E80FF11DEC53FD4F81E06081A5
:1002E0000E94120480E293E00197F1F78091180DCB
:1002F0008F5F8093180D86E00E948C048F7180932D
:10030000190D6091180D40918B0D0E949510FF9171
:10031000EF91BF91AF919F918F917F916F915F917D
:100320004F913F912F910F900BBE0F900FBE0F90EA
:100330001F9018951F920F920FB60F920BB60F9247
:100340001124EF920F932F933F934F935F936F93EB
:100350007F938F939F93AF93BF93EF93FF93DF931D
:10036000CF9300D0CDB7DEB719821A828FE00E94FA
:100370008C04A89582FF07C086E00E948C048F71D0
:100380008093880D2AC183FF28C18091890D9091A7
:100390008A0D019709F002C18BE19DE06CE6AE0188
:1003A0004E5F5F4F9E012F5F3F4F0E940D058823D8
:1003B00009F413C18981882309F40FC12091380EF3
:1003C0003091390E40913A0E50913B0E80911B0DA9
:1003D00090911C0DA0911D0DB0911E0D82179307D9
:1003E000A407B50709F088C08091A4009091A500EA
:1003F0009093170D8093160D1092A5001092A400F3
:100400008091180D882331F48CE390E090932302BF
:10041000809322028091220290912302E0913D0E6E
:1004200020918B0D0A96F0E0B4E0EE0FFF1FBA9515
:10043000E1F7E20FF11DEC5DFD4F2081820F911D70
:100440009093A9008093A800A8950E949110009114
:10045000180DE0908B0D8BE19DE06091880D40912F
:10046000870D2A810E945413082F86E00E948C0475
:100470008F718093870D8430F8F40023E9F0E091C8
:100480003C0E80918B0DF0E0A4E0EE0FFF1FAA95CB
:10049000E1F7E80FF11DEC53FD4F82E060810E940F
:1004A000120480E293E00197F1F78BE19DE0602F69
:1004B00070E00E94090419C00E94FB03E0913C0E09
:1004C00080918B0DF0E074E0EE0FFF1F7A95E1F75D
:1004D000E80FF11DEC53FD4F81E060810E94120492
:1004E00080E293E00197F1F7A8958091180D809331
:1004F0001A0D1092180D71C08091380E9091390E1E
:10050000A0913A0EB0913B0E0097A105B10509F0FC
:1005100064C08091880D853008F45FC0A8950E9462
:1005200091108091380E9091390EA0913A0EB091B1
:100530003B0E20911B0D30911C0D40911D0D5091D3
:100540001E0D82179307A407B50771F080911F0D48
:100550008150823048F42093380E3093390E409306
:100560003A0E50933B0EA8950E94FB03E0913C0E7F
:1005700080918B0DF0E064E0EE0FFF1F6A95E1F7CC
:10058000E80FF11DEC53FD4F81E060810E941204E1
:1005900080E293E00197F1F7A8951FC00E94FB034A
:1005A000E0913C0E80918B0DF0E054E0EE0FFF1FC8
:1005B0005A95E1F7E80FF11DEC53FD4F81E06081A2
:1005C0000E94120480E293E00197F1F7A89586E07B
:1005D0000E948C048F718093870D0F900F90CF91A4
:1005E000DF91FF91EF91BF91AF919F918F917F919B
:1005F0006F915F914F913F912F910F91EF900F90DD
:100600000BBE0F900FBE0F901F901895DF93CF93E6
:1006100000D000D0CDB7DEB789E492E0A0E0B0E032
:1006200089839A83AB83BC83CE01019660E070E03E
:1006300044E050E00E94452488E39EE064E070E0DE
:1006400042E550E00E9445240F900F900F900F90CC
:10065000CF91DF910895EF92FF920F93DF93CF93A5
:10066000CDB7DEB768970FB6F894DEBF0FBECDBF2B
:1006700019821A821B821C820E94B300CE0101964D
:1006800060E070E044E050E00E94352489819A8166
:10069000AB81BC8105E0E02EF12CEC0EFD1E8954EF
:1006A0009240A040B040D1F488E39EE064E070E066
:1006B00042E550E00E94352480E092E00E946B0801
:1006C0002091380E3091390E40913A0E50913B0EE8
:1006D000C701B90140E020E001E018C080E192E0EC
:1006E0000E946B0869817A81C70140E020E001E047
:1006F0000E94F806C7010E946B0880E292E00E9407
:100700006B08C70169E472E040E020E00E94F8064F
:10071000C7010E946B088DE092E00E946B0868960A
:100720000FB6F894DEBF0FBECDBFCF91DF910F9112
:10073000FF90EF9008958AEF90E0909323028093CA
:1007400022020E942B0380913C0E8A3010F4809389
:100750003C0E0E9437040E94FB03E0913C0E809106
:100760008B0DF0E094E0EE0FFF1F9A95E1F7E80F94
:10077000F11DEC53FD4F81E060810E94120485E081
:100780006FE040E020E00E94B0040E94D603109287
:10079000A5001092A40080912202909123029093D0
:1007A000A9008093A8000E94911008951092A500BE
:1007B0001092A4001092A00085E08093A1008FEF1A
:1007C00090E09093A9008093A800E2E7F0E0808198
:1007D000826080837894089594B7977F94BFE0E611
:1007E000F0E090819861908387708860808384B7FF
:1007F000877F84BF089580918B0D8F3030F4809176
:100800008B0D8F5F80938B0D02C010928B0D80E05B
:1008100008959C01862FB9010E9465052C9A2C9899
:1008200080E008951F93182F262F88E06FE140E0A5
:100830000E94B004812F90E090938A0D8093890DDF
:10084000113019F482E066E008C085E060E847E016
:1008500021E00E94B00482E069E00E947D048EE005
:100860006CE00E947D04789480E01F9108950F93BE
:100870001F9384E00E9458040CEF13E0C801019715
:10088000F1F717982C988CE090E00197F1F7179A00
:1008900082E068E00E947D04C8010197F1F781E0E1
:1008A0006FE140E00E949D0480E01F910F91089548
:1008B0000F9A249A95B1936095B994B1976094B9C1
:1008C000239890E59CBD9CB59C7F9CBD9DB59E7F6B
:1008D0009DBD2CB5982F9370922B9CBD9DB5869590
:1008E00086958170982B9DBDEAE6F0E080818C6052
:1008F000808380E28CBBED9A0895806C9FB7F8945A
:1009000028988EBD0DB407FEFDCF6EBD0DB407FE59
:10091000FDCF289A9FBF08958F7380689FB7F89482
:1009200028988EBD0DB407FEFDCF8EBD0DB407FE19
:10093000FDCF8EB5289A9FBF0895FF920F931F9306
:10094000062FF42E0E948C04082310E002C0159597
:100950000795FA94E2F7802F1F910F91FF90089569
:10096000DF92EF92FF920F931F93D82EF62EE42E74
:10097000022F0E948C046F2D6095682310E002C046
:10098000000F111FEA94E2F7F0226F298D2D0E94CB
:100990007D041F910F91FF90EF90DF900895CB01A0
:1009A0000895FC01DA015FB7F894289880E28EBDC3
:1009B0000DB407FEFDCF1EBC0DB407FEFDCF4EB536
:1009C000641730F1942F20E030E01EBC0DB407FE18
:1009D000FDCF8EB52827022E2295207F2025032EBD
:1009E000322F22952F700226269532272327220F99
:1009F000220F220F20258083915011F03196E5CFF0
:100A0000109739F01C92232B21F481E08C9301C0C4
:100A10004068289A5FBF842F0895FF920F931F9319
:100A2000CF93DF938C01EA01D901FFB6F89428989F
:100A300080E28EBD0DB407FEFDCF1EBC0DB407FED7
:100A4000FDCF9EB5691708F436C020E030E040E0E5
:100A500050E0692F70E01CC01EBC0DB407FEFDCF36
:100A60008EB5F801E20FF31F80834827042E4295CC
:100A7000407F4025052E542F42954F700426469501
:100A800054274527440F440F440F40252F5F3F4F05
:100A90002617370708F3109729F01C92452B11F4FD
:100AA00081E08C93209741F01EBC0DB407FEFDCF72
:100AB0008EB5888301C09068289AFFBE892FDF9188
:100AC000CF911F910F91FF900895982FFB012FB7A1
:100AD000F894289880E68EBD0DB407FEFDCF9EBD2C
:100AE0000DB407FEFDCF80818EBD915011F031967F
:100AF000F7CF0DB407FEFDCF289A2FBF0895FC0154
:100B0000DA013FB7F894289880E28EBD0DB407FE55
:100B1000FDCF1EBC0DB407FEFDCF2EB56217A0F0B1
:100B2000922F1EBC0DB407FEFDCF8EB58083915071
:100B300011F03196F6CF109741F01EBC0DB407FEB0
:100B4000FDCF8EB58C9301C02068289A3FBF822FBD
:100B50000895833309F080E0089583E30895E82F32
:100B6000F0E0EE0FFF1FE057F14F20813181C90106
:100B70000895E82FF0E0EE0FFF1FE057F14F1182CC
:100B8000108208959B01AC01529A53985A9A5B9A2D
:100B900064E0220F331F441F551F6A95D1F760E0B0
:100BA00072E18AE790E00E94852321503040109244
:100BB000CD002093CC0080E48093C80088E9809326
:100BC000C90086E08093CA00789408959B01AC0127
:100BD000689A6998709A719A74E0220F331F441FC3
:100BE000551F7A95D1F760E072E18AE790E00E94A4
:100BF0008523215030401092C5002093C40080E42A
:100C00008093C00088E98093C10086E08093C20091
:100C100078940895FC0180918D0E8823D1F4F0938F
:100C20008F0EE0938E0E60938D0E2091920E309178
:100C3000930E808190E0822793279093930E809368
:100C4000920E80818093CE008091C9008062809353
:100C5000C90080918D0E8823E1F70895FC018091F1
:100C60008A0E8823D1F4F0938C0EE0938B0E609360
:100C70008A0E2091900E3091910E808190E0822713
:100C800093279093910E8093900E80818093C6005D
:100C90008091C10080628093C10080918A0E882378
:100CA000E1F70895DF93CF930F92CDB7DEB7898335
:100CB000CE01019661E00E942E060F90CF91DF9148
:100CC0000895DF93CF930F92CDB7DEB78983CE011E
:100CD000019661E00E940A060F90CF91DF9108957E
:100CE0001F920F920FB60F920BB60F9211242F93F3
:100CF0003F938F939F93EF93FF93E0918E0EF0912C
:100D00008F0E3196F0938F0EE0938E0E3197809177
:100D10008D0E815080938D0E80918D0E882391F0E1
:100D20008091920E9091930E2181332727FD30956B
:100D3000282739273093930E2093920E8181809338
:100D4000CE0005C08091C9008F7D8093C900FF91BE
:100D5000EF919F918F913F912F910F900BBE0F902C
:100D60000FBE0F901F9018951F920F920FB60F9203
:100D70000BB60F9211242F933F938F939F93EF9372
:100D8000FF93E0918B0EF0918C0E3196F0938C0EC8
:100D9000E0938B0E319780918A0E815080938A0E5A
:100DA00080918A0E882391F08091900E9091910EFF
:100DB0002181332727FD3095282739273093910E3D
:100DC0002093900E81818093C60005C08091C10060
:100DD0008F7D8093C100FF91EF919F918F913F9103
:100DE0002F910F900BBE0F900FBE0F901F90189574
:100DF000BF92CF92DF92EF92FF920F931F93DF93F8
:100E0000CF93CDB7DEB72C970FB6F894DEBF0FBEE9
:100E1000CDBF6C01FB01B42EE22E77FD02C0FF2492
:100E200008C0F095E195FF4F8DE2D6018C93FF2429
:100E3000F39440E08E010F5F1F4F10C0200F311F51
:100E4000CF016AE070E00E947223805DD9018C932B
:100E5000CF016AE070E00E947223FB01242F30E092
:100E60004F5FEA30F10554F7020F131F8E2F805D9C
:100E7000F8018083642FCE01019620E305C0FC01B8
:100E8000E60FF11D20836F5FE616C8F76B15B8F308
:100E9000862F90E09E012F5F3F4FF901E80FF91F69
:100EA00010820197D901A80FB91F019640E050E0C8
:100EB0008C012E2D30E07EE214C0C801841B950BFE
:100EC0008217930729F4F601EF0DF11D7083F39457
:100ED000F601EF0DF11D8C918083F3944F5F5F4F0E
:100EE0001197461750F3F601EF0DF11D1082C60160
:100EF0002C960FB6F894DEBF0FBECDBFCF91DF9119
:100F00001F910F91FF90EF90DF90CF90BF900895C9
:100F10004F925F926F927F928F929F92AF92BF9209
:100F2000CF92DF92EF92FF920F931F93DF93CF93B5
:100F3000CDB7DEB72C970FB6F894DEBF0FBECDBF8E
:100F40003C016A017B01422E502E77FD02C099249C
:100F50000DC0F094E094D094C094C11CD11CE11C4D
:100F6000F11C8DE2F30180839924939488245E011F
:100F70000894A11CB11C19C00A0D1B1DC701B601A4
:100F80002AE030E040E050E00E94A723605DF801D5
:100F90006083C701B6012AE030E040E050E00E94E3
:100FA000A723C901DA016C017D01082D10E08394AB
:100FB000FAE0CF16D104E104F104F4F6A00EB11E5C
:100FC0008C2D805DF5018083482DCE01019620E3B4
:100FD00005C0FC01E40FF11D20834F5F5416C8F7D4
:100FE0004415B8F3842F90E09E012F5F3F4FF90125
:100FF000E80FF91F10820197D901A80FB91F0196B8
:1010000020E030E0BC01052D10E05EE214C0CB0111
:10101000821B930B8017910729F4F301E90DF11D51
:1010200050839394F301E90DF11D8C918083939487
:101030002F5F3F4F1197241750F3F301E90DF11D76
:101040001082C3012C960FB6F894DEBF0FBECDBF41
:10105000CF91DF911F910F91FF90EF90DF90CF9094
:10106000BF90AF909F908F907F906F905F904F90C8
:101070000895DC010D900020E9F71197A81BB90B2A
:101080006A2F0E942E060895EF92FF920F93DF932E
:10109000CF93CDB7DEB72A970FB6F894DEBF0FBE59
:1010A000CDBFBC017E010894E11CF11CC70140E0EA
:1010B00020E001E00E94F806C7010E9439082A9644
:1010C0000FB6F894DEBF0FBECDBFCF91DF910F9169
:1010D000FF90EF900895DC010D900020E9F7119743
:1010E000A81BB90B6A2F0E940A060895CF92DF92BF
:1010F000EF920F93DF93CF93CDB7DEB72A970FB65A
:10110000F894DEBF0FBECDBFAB01BC016E010894E9
:10111000C11CD11CC60120E000E0EE24E3940E9433
:101120008807C6010E946B082A960FB6F894DEBFA6
:101130000FBECDBFCF91DF910F91EF90DF90CF9099
:101140000895EF92FF920F93DF93CF93CDB7DEB761
:101150002A970FB6F894DEBF0FBECDBFBC017E014B
:101160000894E11CF11CC70140E020E001E00E946E
:10117000F806C7010E946B082A960FB6F894DEBFE6
:101180000FBECDBFCF91DF910F91FF90EF900895EB
:10119000809881988298839886E880937A0080E48A
:1011A00080937C000895806480937C0086E880931F
:1011B0007A0080917A00806480937A0080917A002E
:1011C00084FFFCCF2091780030917900C901089507
:1011D000E82F80917A0E8E1709F43FC08091800E1F
:1011E0008E17D9F18091740E813118F080E18093CF
:1011F000740E2091750E3091760E8091770E90913D
:10120000780E4FEF5FE1DA01A81BB90BA217B30705
:1012100050F48091770E9091780E481B590B5093A3
:10122000760E4093750E8091770E9091780E23E0A4
:10123000880F991F2A95E1F79093650380936403C3
:101240008091740EE81748F4F0E06052714DEE0F93
:10125000FF1FEF56F24F718360830895109285004F
:1012600010928400089580E090E020EE3EE2FC01C0
:10127000EE0FFF1FEF56F24F31832083019680312E
:101280009105A9F7259A2D9A82E08093800088E144
:10129000809381008091800080688093800080919D
:1012A00081008160809381008FEF9FEF9093870092
:1012B0008093860080916F00816080936F007894A6
:1012C00008951F920F920FB60F920BB60F92112432
:1012D0002F933F934F935F938F939F93EF93FF933E
:1012E0008091790E882371F4809188009091890013
:1012F0002091640330916503820F931F90938700C0
:101300008093860050918E0D8091740E581708F0CE
:101310008CC080917A0E851791F5E0917D0EF09149
:101320007E0E43E0EE0FFF1F4A95E1F740918F0DCF
:1013300080917B0E481780F480917F0EE42FF0E0BF
:10134000E80FF11DEE0FFF1FEC56F14F0190F081F9
:10135000E02DE052F14D0CC080917C0E823061F4A2
:1013600080917B0E90E0242F30E08217930724F0C9
:101370004F5F40938F0D38C010928F0D35C0809114
:10138000800E8517E1F5E091830EF091840E23E045
:10139000EE0FFF1F2A95E1F74091900D8091810E8D
:1013A000481780F48091850EE42FF0E0E80FF11DDE
:1013B000EE0FFF1FEC56F14F0190F081E02DE0524F
:1013C000F14D0CC08091820E823061F48091810ECB
:1013D00090E0242F30E08217930724F04F5F409372
:1013E000900D02C01092900D80916403909165035E
:1013F000E81BF90BF0938D0DE0938C0D12C0E52FD7
:10140000F0E0EE0FFF1FEF56F24F808191812091A7
:10141000640330916503821B930B90938D0D809331
:101420008C0D5F5F50938E0D0FC08091750E909163
:10143000760E53E0880F991F5A95E1F790938D0D22
:1014400080938C0D10928E0D8091790E20918C0DD1
:1014500030918D0D882329F43093890020938800E2
:1014600012C08091880090918900820F931F909301
:101470008700809386008091640390916503909328
:10148000890080938800FF91EF919F918F915F91E8
:101490004F913F912F910F900BBE0F900FBE0F9069
:1014A0001F901895519A509A599A589AE9EBF0E082
:1014B00080818360808380E28093B80084E08093A1
:1014C000BC00089584EA8093BC00089584E9809369
:1014D000BC00089520E030E002C02F5F3F4F8091B4
:1014E000BC0087FD06C083E228323807B1F780E0F0
:1014F000089580E02852334208F481E008958093F3
:10150000BB0084E88093BC000895813029F4809169
:10151000BC008F70806C04C08091BC008F708068AC
:101520008093BC0008958091BB0008958091B9001C
:101530000895EF92FF920F931F93CF93DF93182F8D
:10154000E62E042FF52E84EA8093BC000E946A0ADE
:101550001093BB0084E88093BC000E946A0A8091CB
:10156000B9008871B1F4802F9F2D9C01E90110E032
:1015700004E808C089918093BB000093BC000E94DE
:101580006A0A1F5F1E15B0F384E98093BC0081E0F6
:1015900004C084E98093BC0080E0DF91CF911F916B
:1015A0000F91FF90EF9008950F931F93182F062F20
:1015B00084EA8093BC000E946A0A1093BB0014E87E
:1015C0001093BC000E946A0A8091B900887159F09A
:1015D0000093BB001093BC000E946A0A84E98093C8
:1015E000BC0081E004C084E98093BC0080E01F91CE
:1015F0000F910895FF920F931F93182F062FF42E2B
:1016000084EA8093BC000E946A0A1093BB0014E82D
:101610001093BC000E946A0A8091B900887189F019
:101620000093BB001093BC000E946A0AF092BB00BA
:101630001093BC000E946A0A84E98093BC0081E098
:1016400004C084E98093BC0080E01F910F91FF905B
:101650000895CF92DF92EF92FF921F93CF93DF9383
:10166000182FF62E6A0184EA8093BC000E946A0A51
:101670001F5F1093BB0084E88093BC000E946A0A3D
:101680008091B900887159F510E0CF2DD0E02197F5
:101690000CC081E00E94850A0E946A0A8091BB000A
:1016A000F70180830E946A0A1F5F812F90E0760114
:1016B000E80EF91E8C179D0764F380E00E94850AEE
:1016C0000E946A0A8091BB00F70180830E946A0A27
:1016D00084E98093BC000E946A0A81E006C084E924
:1016E0008093BC000E946A0A80E0DF91CF911F9135
:1016F000FF90EF90DF90CF9008950F931F93DF93AB
:10170000CF9300D0CDB7DEB781E489831A8282E41B
:1017100061E08E010F5F1F4FA8010E94990A81307E
:1017200011F080E006C082E462E0A8010E94290B6B
:1017300081E00F900F90CF91DF911F910F9108954D
:101740000F931F93DF93CF9300D0CDB7DEB781E423
:1017500089831A8282E461E08E010F5F1F4FA80126
:101760000E94990A813029F482E462E0A8010E9473
:10177000290B998180E02A8130E0282B392BC9017F
:101780000F900F90CF91DF911F910F9108952F929D
:101790003F924F925F926F927F928F929F92AF9201
:1017A000BF92CF92DF92EF92FF920F931F93DF933E
:1017B000CF93CDB7DEB72E970FB6F894DEBF0FBE2E
:1017C000CDBFFE0131968AE0DF011D928A95E9F7CF
:1017D0008EEE64EF4EE20E94FA0A813009F588E04D
:1017E00092E028EC30E0F9013197F1F70197D9F751
:1017F0008EEE66EF0E94D40A813079F48EEE62E0BC
:10180000AE014F5F5F4F0E94290B998180E02A81D2
:10181000022F10E0082B192B09C086E693E002C0C6
:101820008DE693E00E946B0800E010E08EEE64EF1E
:1018300044EF0E94FA0A8130D1F588E29AE028EC60
:1018400030E0F9013197F1F70197D9F78EEE66EFA5
:101850000E94D40A813041F58EEE63E0AE014F5F05
:101860005F4F0E94290B898190E0A0E0B0E02C013D
:10187000332422248B8190E0A0E0B0E0282A392A8A
:101880004A2A5B2A9A8180E0AA2797FDA095BA2F61
:10189000282A392A4A2A5B2A45E0559447943794E6
:1018A00027944A95D1F70AC084E793E002C08BE7FA
:1018B00093E00E946B08222433242101B801882779
:1018C00077FD8095982F2091C10D3091C20D40E099
:1018D00050E0621B730B840B950B2091BF0D309170
:1018E000C00D40E050E00E943F237B018C013FE0AF
:1018F00015950795F794E7943A95D1F76091C90D3E
:101900007091CA0D882777FD8095982F2BE0660F80
:10191000771F881F991F2A95D1F72091CB0D309101
:10192000CC0D442737FD4095542F2E0D3F1D401FF1
:10193000511F0E94A72359016A01AE0CBF1CC01E93
:10194000D11E88E090E0A0E0B0E0A80EB91ECA1E4B
:10195000DB1ED601C50114E0B595A795979587952F
:101960001A95D1F79093B20D8093B10D88E590EF61
:10197000AFEFBFEFA80EB91ECA1EDB1EC601B50130
:10198000A60195010E943F233B014C01ACE09594D8
:10199000879477946794AA95D1F72091BB0D3091E5
:1019A000BC0D442737FD4095542FC601B5010E9458
:1019B0003F237B018C01FDE015950795F794E79493
:1019C000FA95D1F782E090E0A0E0B0E0E80EF91ED1
:1019D0000A1F1B1F2091C30D3091C40D442737FDF2
:1019E0004095542FC401B3010E943F23BC019927A5
:1019F00077FD9095892FE60EF71E081F191F52E0FC
:101A000015950795F794E7945A95D1F780E090E8FB
:101A1000A0E0B0E0E80EF91E0A1F1B1F2091BD0DCB
:101A20003091BE0D40E050E0C801B7010E943F2355
:101A3000DC01CB014FE0B695A795979587954A9520
:101A4000D1F78B879C87AD87BE872091B90D3091E8
:101A5000BA0D442737FD4095542FC601B5010E94A9
:101A60003F237B018C013BE015950795F794E794A4
:101A70003A95D1F78091B70D9091B80DAA2797FDAF
:101A8000A095BA2F22E0880F991FAA1FBB1F2A9585
:101A9000D1F7E80EF91E0A1F1B1F2091C50D3091CA
:101AA000C60D442737FD4095542FC401B3010E9451
:101AB0003F23ABE09595879577956795AA95D1F7E4
:101AC000E60EF71E081F191FEE0CFF1C001F111F4A
:101AD0002E183F08400A510AC201B1012AE638E136
:101AE00040E050E00E943F2397FD0FC0660F771F34
:101AF000881F991F2B853C854D855E850E94852317
:101B0000C901DA015C016D010CC02B853C854D8556
:101B10005E850E94852359016A01AA0CBB1CCC1C5E
:101B2000DD1C5527D7FC5A954D2D3C2D2B2DCA0178
:101B3000B9010E943F232EED3BE040E050E00E94BF
:101B40003F237B018C01C601B50123E433EE4FEF47
:101B50005FEF0E943F23BC01992777FD9095892F65
:101B60006153714F8F4F9F4F78011127F7FC1095EC
:101B7000012F6E0D7F1D801F911F24E09595879585
:101B8000779567952A95D1F76A0D7B1D8C1D9D1D54
:101B90006093B30D7093B40D8093B50D9093B60D13
:101BA00081E02E960FB6F894DEBF0FBECDBFCF9169
:101BB000DF911F910F91FF90EF90DF90CF90BF903A
:101BC000AF909F908F907F906F905F904F903F90DD
:101BD0002F90089582E893E00E946B088091B10DE8
:101BE0009091B20D6AE070E00E947223882777FD21
:101BF0008095982F0E94760889E893E00E946B08F0
:101C00008091B10D9091B20D6AE070E00E94722354
:101C1000AA2797FDA095BA2FBC01CD010E94760896
:101C20008BE893E00E946B088091B10D9091B20D0A
:101C300008958EE893E00E946B086091B30D709157
:101C4000B40D8091B50D9091B60D0E9476088BE889
:101C500093E00E946B086091B30D7091B40D809178
:101C6000B50D9091B60D08950F931F93DF93CF9309
:101C7000CDB7DEB72A970FB6F894DEBF0FBECDBF43
:101C80008E010F5F1F4F8AE0F80111928A95E9F7E4
:101C90008EEE64EF4EE20E94FA0A813011F080E08D
:101CA000DAC18EEE6AEA0E94D40A8EEE62E0A801E2
:101CB0000E94290B813081F4898190E0A0E0B0E09E
:101CC000BA2FA92F982F88272A8130E0282B392B6B
:101CD0003093B80D2093B70D8EEE6CEA0E94D40AB3
:101CE0008EEE62E0AE014F5F5F4F0E94290B8130A4
:101CF00081F4898190E0A0E0B0E0BA2FA92F982F5D
:101D000088272A8130E0282B392B3093BA0D209375
:101D1000B90D8EEE6EEA0E94D40A8EEE62E0AE013C
:101D20004F5F5F4F0E94290B813081F4898190E0E1
:101D3000A0E0B0E0BA2FA92F982F88272A8130E0A1
:101D4000282B392B3093BC0D2093BB0D8EEE60EB0E
:101D50000E94D40A8EEE62E0AE014F5F5F4F0E9498
:101D6000290B813081F4898190E0A0E0B0E0BA2FA6
:101D7000A92F982F88272A8130E0282B392B3093E0
:101D8000BE0D2093BD0D8EEE62EB0E94D40A8EEE46
:101D900062E0AE014F5F5F4F0E94290B813081F4FA
:101DA000898190E0A0E0B0E0BA2FA92F982F882772
:101DB0002A8130E0282B392B3093C00D2093BF0DA2
:101DC0008EEE64EB0E94D40A8EEE62E0AE014F5FAD
:101DD0005F4F0E94290B813081F4898190E0A0E05F
:101DE000B0E0BA2FA92F982F88272A8130E0282B1E
:101DF000392B3093C20D2093C10D8EEE66EB0E94FD
:101E0000D40A8EEE62E0AE014F5F5F4F0E94290B55
:101E1000813081F4898190E0A0E0B0E0BA2FA92F51
:101E2000982F88272A8130E0282B392B3093C40D36
:101E30002093C30D8EEE68EB0E94D40A8EEE62E012
:101E4000AE014F5F5F4F0E94290B813081F4898181
:101E500090E0A0E0B0E0BA2FA92F982F88272A8120
:101E600030E0282B392B3093C60D2093C50D8EEE14
:101E70006AEB0E94D40A8EEE62E0AE014F5F5F4FC4
:101E80000E94290B813081F4898190E0A0E0B0E0CC
:101E9000BA2FA92F982F88272A8130E0282B392B99
:101EA0003093C80D2093C70D8EEE6CEB0E94D40AC0
:101EB0008EEE62E0AE014F5F5F4F0E94290B8130D2
:101EC00081F4898190E0A0E0B0E0BA2FA92F982F8B
:101ED00088272A8130E0282B392B3093CA0D209394
:101EE000C90D8EEE6EEB0E94D40A8EEE62E0AE015A
:101EF0004F5F5F4F0E94290B813081F4898190E010
:101F0000A0E0B0E0BA2FA92F982F88272A8130E0CF
:101F1000282B392B3093CC0D2093CB0D85E993E002
:101F20000E946B086091B70D7091B80D882777FDFE
:101F30008095982F0E9476088CE993E00E946B08A8
:101F40006091B90D7091BA0D882777FD8095982F13
:101F50000E9476088CE993E00E946B086091BB0DAB
:101F60007091BC0D882777FD8095982F0E94760888
:101F70008CE993E00E946B086091BD0D7091BE0DDD
:101F800080E090E00E9476088CE993E00E946B0864
:101F90006091BF0D7091C00D80E090E00E947608C6
:101FA0008CE993E00E946B086091C10D7091C20DA5
:101FB00080E090E00E9476088CE993E00E946B0834
:101FC0006091C30D7091C40D882777FD8095982F7F
:101FD0000E9476088CE993E00E946B086091C50D21
:101FE0007091C60D882777FD8095982F0E947608FE
:101FF0008CE993E00E946B086091C70D7091C80D49
:10200000882777FD8095982F0E9476088CE993E0C9
:102010000E946B086091C90D7091CA0D882777FDE9
:102020008095982F0E9476088CE993E00E946B08B7
:102030006091CB0D7091CC0D882777FD8095982FFE
:102040000E9476088CE993E00E946B088BE893E08D
:102050000E946B0881E02A960FB6F894DEBF0FBE8F
:10206000CDBFCF91DF911F910F910895FC01808129
:10207000860F80830895FC01808181958083089577
:10208000FC018081860F80830895FC018081819509
:1020900080830895FC0180819181860F971F918331
:1020A00080830895FC0180819181909581959F4F57
:1020B000918380830895FC0180819181860F971F11
:1020C000918380830895FC01808191819095819511
:1020D0009F4F918380830895FC01882777FD809529
:1020E000982F2081318142815381260F371F481F4D
:1020F000591F20833183428353830895FC018081DB
:102100009181A281B381B095A095909581959F4FC3
:10211000AF4FBF4F80839183A283B3830895279AE3
:1021200008952F9A08952F980895E42FF0E0DF0185
:10213000AC5CBF4E1C92DF01A05EBF4E8C93E45F8F
:10214000FF4E10826093E70D8091DD0D8A3F28F4E9
:102150008091DD0D8F5F8093DD0D6623C1F080914E
:10216000E10D9091E20D66956695262F30E0820F85
:10217000931F9093E20D8093E10D8091E30D909178
:10218000E40D280F391F3093E40D2093E30D809167
:10219000E10D9091E20D855F9140F0F02091E30D0B
:1021A0003091E40D6091E10D7091E20D84E690E0D4
:1021B000AC01249FC001259F900D349F900D1124E8
:1021C0000E945E236093E00D1092E20D1092E10DEB
:1021D0001092E40D1092E30D08951F920F920FB626
:1021E0000F920BB60F921124EF92FF920F931F9351
:1021F0002F933F934F935F936F937F938F939F930F
:10220000AF93BF93EF93FF939091C6009093E50D2A
:102210008091130E8093140E8091120E8093130EF2
:102220008091110E8093120E8091100E8093110EEA
:102230009093100E80910F0E882349F4943209F088
:102240000CC181E080930F0E10920E0E06C18130FA
:1022500009F041C020910E0E253031F58091FA0D24
:10226000823551F48091FB0D8D3401F58091FC0D88
:102270008334E1F482E00BC08734C1F48091FB0D1C
:10228000873451F48091FC0D813481F483E0809394
:102290000F0E10920E0E1AC0833541F48091FC0D82
:1022A000813421F484E0F3CF243170F4E22FF0E0A4
:1022B000E850F24F9083E22FEF5FE0930E0EF0E0D4
:1022C000E850F24F108202C010920F0E10920D0EC5
:1022D00010920C0EC2C08230E1F59D3009F4BBC0F3
:1022E0009C3209F0A9C0F0900C0E83E18F1508F420
:1022F000A3C0E0900D0EE4E0EE1639F0F6E0EF1624
:1023000021F082E0E81609F091C00F2D10E088EF6F
:102310009DE00E94FD23000F111F00591F4EF80180
:1023200091838083F394F0920C0EE8EFFDE090E04F
:1023300080818E3249F40F2D10E0892F90E0875074
:10234000924F0E94FD2367C09F5F3196943181F7C1
:102350006DC0833009F047C09D3009F47CC09C32C9
:1023600009F06AC0F0900C0EF3E1FF1508F464C0A8
:10237000E0900D0E85E0E81608F458C0E6E0EE1592
:1023800020F4F8E0EF1609F051C00F2D10E00A5FBD
:102390001F4F88EF9DE00E94FD239C01000F111F3D
:1023A00000591F4EF80131832083F394F0920C0EF4
:1023B00020E030E0822FF901E850F24FE081EE2377
:1023C000A9F1EE3251F40F2D10E00A5F1F4F90E09B
:1023D0008750924F0E94FD231EC02F5F3F4F243134
:1023E000310541F723C08430B1F59D30A1F19C3215
:1023F00019F5F0900C0EF3E1FF15F0F0E0900D0EE2
:1024000081E0E81699F40F2D10E0065F1F4F88EF6A
:102410009DE00E94FD239C01000F111F00591F4EDB
:10242000F80131832083F394F0920C0E10920E0E7B
:10243000E394E0920D0E11C0A0910E0EEA2FF0E091
:10244000E850F24F9083AF5FA0930E0EB0E0A8501B
:10245000B24F1C9202C010920F0EFF91EF91BF91EC
:10246000AF919F918F917F916F915F914F913F912C
:102470002F911F910F91FF90EF900F900BBE0F9037
:102480000FBE0F901F9018951F920F920FB60F92CC
:102490000BB60F9211242F933F934F935F936F933B
:1024A0007F938F939F93AF93BF93EF93FF93DF93AC
:1024B000CF9300D000D000D0CDB7DEB75091CE0082
:1024C0005093E60D9091F60D9093F70D2091F50D38
:1024D0002093F60D3091F40D3093F50D4091F30DEE
:1024E0004093F40D5093F30D8091F00D823001F57F
:1024F0008091F20D813309F08DC099832A833B834B
:102500004C835D831E82CE0101960E94F92320E058
:1025100030E040E251E40E941B200E94451E6115FC
:10252000710509F475C0709373106093721070C0D8
:102530008091F00D813009F073C08091F20D8231ED
:1025400091F499832A833B834C831D821E82CE01A2
:1025500001960E94FD23009709F45CC090937110CE
:102560008093701057C0873191F499832A833B83FD
:102570004C831D821E82CE0101960E94FD2300978E
:1025800009F448C0909373108093721043C08F3148
:1025900089F499832A833B834C835D831E82CE0119
:1025A00001960E94FD230097A9F1909375108093E6
:1025B000741030C0843289F499832A833B834C831E
:1025C0005D831E82CE0101960E94FD23009711F1CA
:1025D00090937710809376101DC08B32D9F4998335
:1025E0002A833B834C835D831E82CE0101960E9429
:1025F000F92320E030E048EC52E40E941B200E94C6
:10260000451E6115710521F0709379106093781063
:102610001092F00D8091F20D8F5F8093F20D2CC01F
:102620009734B9F42035A9F4323541F44D3489F4A6
:10263000533479F41092F20D81E009C0373449F433
:10264000473439F4513429F41092F20D82E080932A
:10265000F00D8091F60D823B79F48091F50D853A6D
:1026600059F48091F40D853639F45B3429F4F894EB
:1026700080E00E94EC03FFCF2696DEBFCDBFCF9156
:10268000DF91FF91EF91BF91AF919F918F917F91DA
:102690006F915F914F913F912F910F900BBE0F90D3
:1026A0000FBE0F901F901895EF920F93CF93DF936B
:1026B000EC01EE2DF0E0DF01AC5CBF4E6C93DF016E
:1026C000A05EBF4E4C93E45FFF4E20830093E70D66
:1026D00088819981AA81BB818093E90D9093EA0D4D
:1026E000A093EB0DB093EC0D1092DD0D8091E10DF8
:1026F0009091E20D01969093E20D8093E10D0023FD
:10270000C1F08091E10D9091E20D202F2695269544
:1027100030E0820F931F9093E20D8093E10D809142
:10272000E30D9091E40D280F391F3093E40D2093B1
:10273000E30D8091E10D9091E20D855F9140F0F005
:102740002091E30D3091E40D6091E10D7091E20D67
:1027500084E690E0AC01249FC001259F900D349F3A
:10276000900D11240E945E236093E00D1092E20D03
:102770001092E10D1092E40D1092E30D8C818130E6
:1027800009F07DC088E08093DF0D888D998D90934E
:10279000170E8093160EE0E010C0F0E0DF011496F3
:1027A000AA0FBB1FAC0FBD1F8D919C91EE0FFF1F99
:1027B000E85BFF4E91838083E22F8091DF0D2E2F07
:1027C0002F5FE81750F3E093150E8E818F3F39F499
:1027D0008F81882321F08093090D1092DE0D1092D5
:1027E000150E24C0842F90E0FC01EE0FFF1FDF01C7
:1027F000A85BBF4E2D913C91EC56F14F3183208365
:10280000885C914FDC015896EC91F0E0EE0FFF1FD1
:10281000E85BFF4E60817181660F771F842F0E94F5
:10282000E8088091150E8F5F8093150E4091150E6C
:102830008091DF0D4817B0F28E818093D30D8E8189
:10284000E82FF0E08091DF0D9F01280F311D20342B
:1028500031058CF48091DF0DE80FF11D8F8124E1AB
:10286000829FC00111248C5E9940EE0FFF1FEC5631
:10287000F14F9183808381E08093F10D7CC08230A1
:1028800009F079C080E18093DF0D88A599A5909328
:10289000170E8093160EE0E010C0F0E0DF011496F2
:1028A000AA0FBB1FAC0FBD1F8D919C91EE0FFF1F98
:1028B000E85BFF4E91838083E22F8091DF0D2E2F06
:1028C0002F5FE81750F3E093150E8E818F3F39F498
:1028D0008F81882321F08093090D1092DE0D1092D4
:1028E000150E24C0842F90E0FC01EE0FFF1FDF01C6
:1028F000A85BBF4E2D913C91EC56F14F3183208364
:10290000885C914FDC015896EC91F0E0EE0FFF1FD0
:10291000E85BFF4E60817181660F771F842F0E94F4
:10292000E8088091150E8F5F8093150E4091150E6B
:102930008091DF0D4817B0F28E818093D30D8E8188
:10294000E82FF0E08091DF0D9F01280F311D20342A
:1029500031058CF48091DF0DE80FF11D8F8124E1AA
:10296000829FC00111248C5E9940EE0FFF1FEC5630
:10297000F14F918380838091160E8093E80D8091B2
:10298000D10D8B3000F584E08C838091D10D8D8347
:102990001E828091D10D90E02AE130E0829FF0010B
:1029A000839FF00D929FF00D1124EC52F14F178A86
:1029B0006091D10D8AE1689FB00111246C52714F72
:1029C000CE0108960EC08091D10D8C30F0F484E0D9
:1029D0008C838091D10D8D831E82CE01089663EA8F
:1029E00073E00E9426248091160E9091170E99A3F1
:1029F00088A301969093170E8093160E8091D10DA7
:102A00008F5F8093D10D84E2B8C08091D10D8F5F2C
:102A10008093D10D8150853110F01092D10D83E05B
:102A20008C8380910A0D8D838091160E9091170EE4
:102A30009987888701969093170E8093160E809140
:102A40000A0D813188F4893008F062C08330A1F129
:102A5000843030F48130F1F0823009F084C01DC040
:102A6000843009F050C037C0833109F466C0843126
:102A700038F4813109F457C0823109F074C058C06C
:102A8000853109F464C0853108F45CC0863109F0F1
:102A90006AC062C00E831F826AC020E030E090E00E
:102AA00008C0E92FF0E0EC5CFF4E8081280F311D5B
:102AB0009F5F9031B0F31DC020E030E090E008C08F
:102AC000E92FF0E0E05EFF4E8081280F311D9F5F0F
:102AD0009031B0F30EC020E030E090E008C0E92F64
:102AE000F0E0E45FFF4E8081280F311D9F5F903141
:102AF000B0F39093150E64E0369527956A95E1F74B
:102B00003F832E8334C090E005970E94D30828C0ED
:102B1000E82FF0E0EE0FFF1FE25DF14F8081918121
:102B20008051984F1DC0809170109091711018C005
:102B3000809172109091731013C0809174109091D5
:102B400075100EC0809176109091771009C0809119
:102B500078109091791004C080917A1090917B1038
:102B60009F838E8304C08E831F8210920A0D8091F2
:102B70000A0D8F5F80930A0D8CE0DF91CF910F914A
:102B8000EF90089582EB93E00E946B080895CF9335
:102B9000DF9381EE93E00E946B08C0E0D0E085EE09
:102BA00093E00E946B08FE01E05EFF4E808190E0A2
:102BB0000E94A1082196C031D10589F787EE93E0E4
:102BC0000E946B08C0E0D0E085EE93E00E946B08A5
:102BD000FE01EC5CFF4E808190E00E94A1082196EE
:102BE000C031D10589F78EEE93E00E946B08C0E0FA
:102BF000D0E085EE93E00E946B08FE01E45FFF4E9B
:102C0000808190E00E94A1082196C031D10589F70A
:102C100085EF93E00E946B0885EE93E00E946B08BD
:102C200080E090E00E94D3080E94A10885EE93E026
:102C30000E946B0881E090E00E94D3080E94A108E6
:102C400085EE93E00E946B0882E090E00E94D3083A
:102C50000E94A10885EE93E00E946B0883E090E05B
:102C60000E94D3080E94A1088CEF93E00E946B0899
:102C7000C0E0D0E085EE93E00E946B08FE01EE0F0D
:102C8000FF1FE85BFF4E808191810E94A108219681
:102C9000C031D10579F783E094E00E946B08C0E071
:102CA000D0E085EE93E00E946B08FE01EE0FFF1F5F
:102CB000E05CF14F808191810E94A1082196C8308B
:102CC000D10579F78AE094E00E946B088091E70DC6
:102CD00090E00E94A10885EE93E00E946B0880912D
:102CE000E30D9091E40D0E94A10885EE93E00E940F
:102CF0006B088091E10D9091E20D0E94A10885EE94
:102D000093E00E946B088091E00D90E00E94A10882
:102D100085EE93E00E946B088091E90D9091EA0D99
:102D2000A091EB0DB091EC0D0E94A10885EE93E00F
:102D30000E946B088091380E9091390EA0913A0E46
:102D4000B0913B0E0E94A10885EE93E00E946B08B3
:102D50008091E80D90E00E94A10882E194E00E9439
:102D60006B08C0E0D0E085EE93E00E946B08FE01A6
:102D7000EE0FFF1FE059FF4E808191810E94A10854
:102D80002196CB30D10579F789E194E00E946B0858
:102D9000DF91CF9108950F931F93CF93DF938FEF20
:102DA0000E9461068FEF0E94610640E050E020E043
:102DB00030E0F901EC5CFF4E8081480F511D2F5F20
:102DC0003F4F20313105A9F7A4E056954795AA95C4
:102DD000E1F7842F0E94610640E050E020E030E0FF
:102DE000F901E45FFF4E8081480F511D2F5F3F4F77
:102DF00020313105A9F7F5E056954795FA95E1F7A9
:102E0000842F0E946106C0E0D0E08E01000F111FE8
:102E1000085B1F4EF801808191818050984F892F67
:102E20000E946106F801808191810E9461062196CD
:102E3000C031D10551F7DF91CF911F910F910895C6
:102E4000CF93DF938FEF0E9461068FEF0E946106A0
:102E500040E050E020E030E0F901EC5CFF4E808182
:102E6000480F511D2F5F3F4F20313105A9F794E0E6
:102E7000569547959A95E1F7842F0E94610640E0A8
:102E800050E020E030E0F901E45FFF4E8081480F20
:102E9000511D2F5F3F4F20313105A9F785E0569531
:102EA00047958A95E1F7842F0E946106C0E0D0E043
:102EB000FE01EE0FFF1FE85BFF4E80819181805085
:102EC000984F60E170E00E947223862F0E94610695
:102ED0002196C031D10561F7DF91CF9108950F930D
:102EE0001F93DF93CF9300D00F92CDB7DEB78BE166
:102EF00089838BE58A838AE48B838E010F5F1F4F62
:102F0000C80163E00E940A0682E089831A82C80130
:102F100062E00E940A060F900F900F90CF91DF9110
:102F20001F910F9108950F931F93DF93CF9300D0BC
:102F300000D0CDB7DEB78BE189838BE58A838BE345
:102F40008B8388E48C838E010F5F1F4FC80164E080
:102F50000E940A0682E089831A82C80162E00E9408
:102F60000A060F900F900F900F90CF91DF911F9155
:102F70000F9108951F93CF93DF930E946F170E94C4
:102F800093178DE194E00E946B0888E594E00E941D
:102F90006B0886E894E00E946B0889EB94E00E943D
:102FA0006B0888EC94E00E946B0880917A0E803167
:102FB00050F581ED94E00E946B0880917B0E90E0CB
:102FC0000E94A10889ED94E00E946B0880917A0E1E
:102FD00090E001960E94A1088AEE94E00E946B089E
:102FE00080917C0E90E00E94A1088DEE94E00E94FA
:102FF0006B0880917D0E90917E0E0E94A1088FEE4D
:1030000094E00E946B0884EF94E00E946B0880E0DB
:1030100095E00E946B0882E195E00E946B0881E2D6
:1030200095E00E946B0887E295E00E946B088DE2B4
:1030300095E00E946B0883E395E00E946B0880E0B6
:1030400095E00E946B0887E495E00E946B08C0E061
:10305000D0E013E0FE01EC5CFF4E8081819FC00157
:1030600011248B5590400E94A10886E595E00E94AE
:103070006B082196C031D10569F788E595E00E947B
:103080006B08C0E0D0E013E0FE01E05EFF4E8081FF
:10309000819FC00111248B5590400E94A10886E5B4
:1030A00095E00E946B082196C031D10569F788E749
:1030B00095E00E946B08C0E0D0E013E0FE01E05E06
:1030C000FF4E4081FE01EC5CFF4E8081819FC0017C
:1030D000112450E09A01220F331F240F351F821B49
:1030E000930B0E94A10886E595E00E946B0821964B
:1030F000C031D10519F788E995E00E946B08C0E05E
:10310000D0E0FE01E45FFF4E808190E00E94A108C4
:1031100086E595E00E946B082196C031D10589F7BC
:1031200088EB95E00E946B088091E70D90E00E948B
:10313000A10888ED95E00E946B088091E30D9091C5
:10314000E40D0E94A1088AED95E00E946B08809131
:10315000E10D9091E20D0E94A1088CED95E00E9496
:103160006B088091E00D90E00E94A1088EED95E043
:103170000E946B088091160D9091170D0E94A10876
:103180008AED95E00E946B088091220290912302C3
:103190000E94A10880E096E00E946B088091E90DF2
:1031A0009091EA0DA091EB0DB091EC0D0E94A10859
:1031B00082E296E00E946B088091380E9091390E61
:1031C000A0913A0EB0913B0E0E94A10885E296E0D4
:1031D0000E946B088091E80D90E00E94A10886E4AF
:1031E00096E00E946B0885E596E00E946B0880E0FF
:1031F00090E00E94D3080E94A10886E696E00E9413
:103200006B0881E090E00E94D3080E94A1088AE642
:1032100096E00E946B0882E090E00E94D3080E9432
:10322000A1088EE696E00E946B0883E090E00E9481
:10323000D3080E94A10882E796E00E946B0889E704
:1032400096E00E946B088091660090E00E94A108C1
:1032500088E896E00E946B0882E996E00E946B087D
:1032600080913C0E90E00E94A10881EA96E00E94C5
:103270006B0880913D0E90E00E94A10888E896E0DE
:103280000E946B0884EA96E00E946B0810E00FC071
:10329000E12FF0E0EE0FFF1FE85BFF4E8081918190
:1032A0000E94A10886E595E00E946B081F5F80914F
:1032B000DF0D181768F388E896E00E946B0883EB2F
:1032C00096E00E946B088091D30D992787FD909519
:1032D0000E94A10888E896E00E946B0882EC96E0C4
:1032E0000E946B0888ED95E00E946B0880917F0E2C
:1032F00090E00E94A10881ED96E00E946B08809109
:103300007F0E20917B0E90E0820F911D0E94A108FC
:1033100084ED96E00E946B0810E011C080917F0E52
:10332000E80FF11DEE0FFF1FEC56F14F80819181E8
:103330000E94A10886E595E00E946B081F5F8091BE
:103340007B0E181750F4E12FF0E080917F0E9F0163
:10335000280F311D203431050CF387ED96E00E94D3
:103360006B0888ED95E00E946B088091850E90E0D7
:103370000E94A10881ED96E00E946B088091850E65
:103380002091810E90E0820F911D0E94A10884ED92
:1033900096E00E946B0810E011C08091850EE80F46
:1033A000F11DEE0FFF1FEC56F14F808191810E94BD
:1033B000A10886E595E00E946B081F5F8091810E51
:1033C000181750F4E12FF0E08091850E9F01280F2F
:1033D000311D203431050CF388E896E00E946B081B
:1033E000DF91CF911F9108950F93FC010190002070
:1033F000E9F73197E81BF90BDB016D917C918E0F9A
:103400009F1F40E020E001E00E94F8060F91089520
:103410000F93FC0101900020E9F73197E81BF90BAD
:10342000DB016D917C918E0F9F1F40E020E001E059
:103430000E94F8060F9108950F93FC01019000205F
:10344000E9F73197E81BF90BDB016D917C918E0F49
:103450009F1F40E020E001E00E94F8060F910895D0
:103460000F93DC010D900020E9F71197A81BB90B11
:10347000FB016081772767FD70958A0F9B1F40E0F5
:1034800020E001E00E94F8060F9108950F93FC01DF
:1034900001900020E9F73197E81BF90BDB016C91F3
:1034A0008E0F9F1F70E040E020E001E00E94F806D0
:1034B0000F9108958F929F92AF92BF92CF92DF9219
:1034C000EF92FF920F931F93DF93CF93CDB7DEB7A9
:1034D000A0970FB6F894DEBF0FBECDBF282F19827C
:1034E0004091CE0D9091CD0DA92FB0E0FD01ED5290
:1034F000F34FE081BE2EB40E8091860E882319F41E
:1035000081E08093860E233309F46AC0243338F4B3
:10351000213309F4ACC0223309F0BCC013C02633F8
:1035200029F1283321F0243309F0B4C060C04423CA
:1035300011F0415012C0A252B34F8C918150809330
:10354000CE0D10C0242F30E0A252B34F8C9190E0EA
:1035500001972817390724F44F5F4093CE0D02C01E
:103560001092CE0DB090CE0DBE0E94C0AB2DB0E03B
:10357000FD01E555F84FE081E230F9F0E33030F439
:10358000EE23D9F0E13009F085C008C0E430F9F04D
:10359000E430E8F0E53009F07DC022C0AA0FBB1F7F
:1035A000A451B84FED91FC9180819181A281B381AA
:1035B0008C509E4FAF4FBF4F4BC0AA0FBB1FA451A3
:1035C000B84FED91FC91808191810A9630C0AA0F8D
:1035D000BB1FA451B84FED91FC9180818F5F45C016
:1035E0009A3010F49F5F46C01092CD0D49C0AB2DAC
:1035F000B0E0FD01E555F84FE081E23079F0E330CD
:1036000030F4EE2359F0E13009F044C013C0E43047
:1036100021F1E43010F1E530E9F529C0AA0FBB1F14
:10362000A451B84FED91FC91808191810A979183CB
:10363000808330C0AA0FBB1FA451B84FED91FC91FD
:1036400080819181A281B381845F9140A040B0408C
:1036500080839183A283B3831DC0AA0FBB1FA45193
:10366000B84FED91FC9180818150808313C09923E4
:1036700021F091509093CD0D03C08AE08093CD0D41
:103680001092CE0DE091CD0DF0E0ED52F34FB080F1
:10369000B092CF0D0B2D10E02091CF0D8091860EB2
:1036A00090E0820F911D0197081719074CF0809147
:1036B000860E2B2D281B822F8F5F8093CF0D04C089
:1036C000B21610F4B092CF0D8FEE96E00E946B0808
:1036D000E091CD0DF0E0ED52F34F208181E090E0DC
:1036E000821B9109800F911F0E94A1088AED95E02D
:1036F0000E946B08E091CD0DF0E0E252F34F808123
:1037000090E00E94A10883EF96E00E946B08E09190
:10371000CD0DF0E0EE0FFF1FE354F34F8081918158
:103720000E946B0885EF96E00E946B088AEF96E096
:103730000E946B08E091CD0DF0E0EE0FFF1FE35407
:10374000F34F6081718188ED9FE00E94262400E0A4
:1037500010E0C8018C52914F6CED75E00E94262458
:10376000065E1F4F31E00430130799F7A090CF0D8C
:103770007E010894E11CF11CEAE18E2E912C89C097
:103780001982BA1429F4C70162E177E00E941B2470
:103790008601000F111FF801E852F44F608171811A
:1037A000C7010E941B24C70164E177E00E941B242B
:1037B000F601E555F84FE081E23001F1E33028F4FD
:1037C000EE2351F0E130C1F510C0E43039F1E430BE
:1037D000F0F0E53089F52BC00451184FF8016081F5
:1037E0007181C7010E94081A27C00451184FF801BF
:1037F00060817181C7010E94F4191EC00451184FE5
:10380000F80160817181C7010E941C1A15C0045122
:10381000184FF80160817181C7010CC00451184F25
:10382000F80160817181C7010E94301A05C0C7018B
:103830006DEC7DE00E94461A86E197E00E946B08DD
:103840008091CF0D9601281B3109C9010E94A10862
:1038500083EF96E00E946B08C7010E946B088AE123
:1038600097E00E946B088091CF0DF601E81BF109EB
:10387000EA30F1056CF4188EE89DC001E99D900DC9
:10388000F89D900D11248C52914FB7010E9426246F
:10389000A394CA2CDD242091860E8091CF0D90E058
:1038A000820F911DC816D906A4F430E43A1588F0A9
:1038B000E091CD0DF0E0DF01A252B34F2C91ED521B
:1038C000F34F808190E0820F911DC816D9060CF449
:1038D00057CF8AEF96E00E946B08A0960FB6F89437
:1038E000DEBF0FBECDBFCF91DF911F910F91FF9033
:1038F000EF90DF90CF90BF90AF909F908F90089502
:10390000CF92DF92EF92FF920F931F93CF93DF93AB
:103910001092D00D1092D20D80E090E02AE130E0BC
:10392000829FF001839FF00D929FF00D1124EC52C5
:10393000F14F108201968A30910591F7279A2F9ABC
:1039400080E090E0FC01EE0FFF1FE85BFF4E11826C
:103950001082019680319105A9F780E090E020E87F
:103960000FB6F89420936100809361000FBE8091A0
:103970006600875F80936600399A419A579A5F9AEA
:103980006B9A739804B603FC03C081E08093EF0D3B
:103990001092EF0D26982E9A60E076E980E090E094
:1039A0000E94C2058DE197E00E946B0882EB93E0D4
:1039B0000E946B0860E875E280E090E00E94E605F6
:1039C0000E94520A0E94C8080E949B030E94330969
:1039D00080E00E945A1ACC24CA9401E093E0F92EA8
:1039E00084E0E82EC4ECD9E012E0D12E9091090DCC
:1039F000C092090D9F3F09F45AC08091DE0D8823C3
:103A000009F055C0992309F452C0892F0E945A1A0F
:103A100080913F0E882309F110923F0E8BE497E0CE
:103A20000E946B0820E030E0F901EE0FFF1FE85B19
:103A3000FF4E80819181F901EE0FFF1FE05CF14F95
:103A4000918380832F5F3F4F2830310569F70E94B3
:103A5000060385E697E00E946B088091890E882313
:103A6000C1F01092890E83E797E00E946B08F092F4
:103A70007A0E10927F0EE092800E1092850ED093F7
:103A8000730EC093720E0E94060385E697E00E94B3
:103A90006B088091880E882341F01092880E0E9456
:103AA000060385E697E00E946B080093DE0DA8955B
:103AB0008091E60D882371F48091ED0D813051F0F5
:103AC0008091F10D813009F0D7C08091EE0D8530E5
:103AD00009F0D2C01091E60D1092E60D133619F4DC
:103AE000D092EE0D04C0123429F4F092EE0D009342
:103AF000ED0D52C01D3619F41092EE0DF8CF1636AA
:103B0000C1F420E030E0F901EE0FFF1FE85BFF4E4B
:103B100080819181F901EE0FFF1FE05CF14F9183ED
:103B200080832F5F3F4F2830310569F70E940603DD
:103B300033C0133721F0812F80538A3028F400934B
:103B4000EE0D1092ED0D28C0133529F40E940603E6
:103B500088E897E01FC0123619F40E94AA001CC022
:103B6000153739F48091ED0D902F981B9093ED0D42
:103B700013C0123759F40E94931784E997E00E940A
:103B80006B08F89480E00E94EC03FFCF193421F415
:103B900082EB93E00E946B088091EE0D823009F475
:103BA00063C0833030F4882359F0813009F064C059
:103BB0000AC0833009F45BC0843009F05DC05AC08C
:103BC0000E94BA1759C0812F0E945A1A80913F0E45
:103BD000882309F110923F0E8BE497E00E946B0856
:103BE00020E030E0F901EE0FFF1FE85BFF4E80811F
:103BF0009181F901EE0FFF1FE05CF14F918380830B
:103C00002F5F3F4F2830310569F70E94060385E694
:103C100097E00E946B088091890E8823C1F0109272
:103C2000890E83E797E00E946B08F0927A0E10925B
:103C30007F0EE092800E1092850ED093730EC0938B
:103C4000720E0E94060385E697E00E946B08809141
:103C5000880E882389F01092880E0E94060385E65C
:103C600097E00E946B0808C00E94C71505C00E941B
:103C7000201702C00E94CB161E99B8CE80EA97E0AA
:103C80000E946B080E94AA00B1CEEF92FF920F93A0
:103C90001F937B018C0120E030E040E05FE40E9454
:103CA000152188238CF0C801B70120E030E040E006
:103CB0005FE40E94BD1F0E9445219B01AC01205082
:103CC00030404040504806C0C801B7010E9445211D
:103CD0009B01AC01B901CA011F910F91FF90EF90B8
:103CE0000895A0E0B0E0E7E7FEE10C94C223DC0118
:103CF0002B01FA019C91923008F439C1EB018881C3
:103D0000823008F433C1943069F4843009F02FC153
:103D100011969C9111978981981709F428C1ABE0FD
:103D2000BDE025C1843009F421C18230A9F492306C
:103D300009F01DC19A01AD0188E0EA010990AE01C8
:103D4000E90109929E018150C1F7E2018981119632
:103D50009C918923818308C1923009F407C112968E
:103D60002D903C901397EB018A819B811496AD9026
:103D7000BD90CD90DC901797EC80FD800E811F8167
:103D80009101281B390BB90137FF04C0662777273B
:103D9000621B730B603271050CF061C012161306C2
:103DA0006CF537014801062E04C0969487947794E9
:103DB00067940A94D2F721E030E040E050E004C07C
:103DC000220F331F441F551F6A95D2F721503040F0
:103DD000404050402E213F214023512321153105E1
:103DE0004105510521F021E030E040E050E079014B
:103DF0008A01E628F728082919293CC0232BD1F18C
:103E0000260E371E35014601062E04C0969487946F
:103E1000779467940A94D2F721E030E040E050E0D4
:103E200004C0220F331F441F551F6A95D2F721503B
:103E30003040404050402A213B214C215D2121153A
:103E400031054105510521F021E030E040E050E02E
:103E500059016A01A628B728C828D9280BC082159D
:103E600093052CF01C01AA24BB24650103C0EE2499
:103E7000FF24870111969C91D20111968C9198177D
:103E800009F445C0992339F0A80197012A193B0983
:103E90004C095D0906C0A60195012E193F09400B8A
:103EA000510B57FD08C0118233822282248335834F
:103EB000468357831DC081E0818333822282882715
:103EC0009927DC01821B930BA40BB50B848395838C
:103ED000A683B7830DC0220F331F441F551F2483B1
:103EE00035834683578382819381019793838283AD
:103EF0002481358146815781DA01C9010197A109E1
:103F0000B1098F5F9F4FAF4FBF4328F30BC0918321
:103F100033822282EA0CFB1C0C1D1D1DE482F582FB
:103F20000683178383E0808324813581468157810E
:103F300057FF1AC0C901AA2797FDA095BA2F817013
:103F40009070A070B0705695479537952795822B45
:103F5000932BA42BB52B84839583A683B78382816F
:103F60009381019693838283DF0101C0D201CD0149
:103F7000CDB7DEB7E2E10C94DE23A0E2B0E0E3ECE3
:103F8000FFE10C94CE2369837A838B839C832D83FA
:103F90003E834F835887E9E0EE2EF12CEC0EFD1E98
:103FA000CE010196B7010E946E228E010F5E1F4F57
:103FB000CE010596B8010E946E228A8991E0892778
:103FC0008A8BC701B801AE01475E5F4F0E94711E28
:103FD0000E949921A096E6E00C94EA23A0E2B0E0CA
:103FE000E4EFFFE10C94CE2369837A838B839C8377
:103FF0002D833E834F835887F9E0EF2EF12CEC0E92
:10400000FD1ECE010196B7010E946E228E010F5E49
:104010001F4FCE010596B8010E946E22C701B8015C
:10402000AE01475E5F4F0E94711E0E949921A096CB
:10403000E6E00C94EA23A0E2B0E0E1E2F0E20C94C6
:10404000C22369837A838B839C832D833E834F8332
:104050005887CE010196BE01675F7F4F0E946E2296
:10406000CE010596BE016F5E7F4F0E946E2299853C
:10407000923088F089898230C8F0943019F4823007
:1040800051F404C0843029F4923081F48BE09DE037
:10409000C6C0923049F420E09A858A89981321E0BD
:1040A0002A87CE010996BBC0823049F420E09A8568
:1040B0008A89981321E02A8BCE014196B0C02D84C5
:1040C0003E844F8458886D887E888F88988CEE2433
:1040D000FF248701AA24BB24650140E050E060E092
:1040E00070E0E0E0F0E0C10181709070892BE9F0B0
:1040F000E60CF71C081D191D9A01AB012A0D3B1D8A
:104100004C1D5D1D80E090E0A0E0B0E0E614F704F7
:104110000805190520F481E090E0A0E0B0E0BA01C4
:10412000A901480F591F6A1F7B1FAA0CBB1CCC1C7E
:10413000DD1C97FE08C081E090E0A0E0B0E0A82A76
:10414000B92ACA2ADB2A3196E032F10549F0660C19
:10415000771C881C991C5694479437942794C3CF96
:10416000FA85EA892B893C898B859C85280F391F24
:104170002E5F3F4F17C0CA0181709070892B61F08C
:1041800016950795F794E79480E090E0A0E0B0E8FA
:10419000E82AF92A0A2B1B2B7695679557954795A0
:1041A0002F5F3F4F77FDE7CF0CC0440F551F661FB1
:1041B000771F17FD4160EE0CFF1C001F111F2150DF
:1041C0003040403090E0590790E0690790E479076B
:1041D00060F32B8F3C8FDB01CA018F779070A0704A
:1041E000B07080349105A105B10561F447FD0AC0A6
:1041F000E114F1040105110529F0405C5F4F6F4F98
:104200007F4F40781A8EFE1711F081E08A8F4D8F14
:104210005E8F6F8F78A383E0898FCE0149960E94CD
:104220009921A096E2E10C94DE23A8E1B0E0EBE155
:10423000F1E20C94CE2369837A838B839C832D8354
:104240003E834F83588789E0E82EF12CEC0EFD1E4B
:10425000CE010196B7010E946E228E010F5E1F4FA4
:10426000CE010596B8010E946E228985823040F009
:104270008989823028F0C701B8010E94E62201C076
:104280008FEF6896E6E00C94EA23ACE0B0E0EBE454
:10429000F1E20C94D22369837A838B839C83CE01D1
:1042A0000196BE016B5F7F4F0E946E228D8182302E
:1042B00061F1823050F1843021F48E81882351F1F4
:1042C0002EC02F81388537FD20C06E812F313105FA
:1042D0001CF06623F9F023C08EE190E0821B930B63
:1042E00029853A854B855C8504C056954795379559
:1042F00027958A95D2F76623B1F050954095309571
:1043000021953F4F4F4F5F4F0EC020E030E040E01F
:1043100050E009C02FEF3FEF4FEF5FE704C020E010
:1043200030E040E050E8B901CA012C96E2E00C947C
:10433000EE23DF92EF92FF920F931F93FC01E48034
:10434000F58006811781D1808081823048F480E039
:1043500090E0A0E1B0E0E82AF92A0A2B1B2BA5C0C7
:10436000843009F49FC0823021F4EE24FF248701B9
:1043700005C0E114F1040105110519F4E0E0F0E0D5
:1043800096C0628173819FEF623879070CF05BC041
:1043900022E83FEF261B370B2A3131052CF020E0B5
:1043A00030E040E050E02AC0B801A701022E04C06E
:1043B00076956795579547950A94D2F781E090E0F6
:1043C000A0E0B0E004C0880F991FAA1FBB1F2A9568
:1043D000D2F70197A109B1098E219F21A023B12312
:1043E0000097A105B10521F081E090E0A0E0B0E0E8
:1043F0009A01AB01282B392B4A2B5B2BDA01C9011F
:104400008F779070A070B07080349105A105B105D0
:1044100039F427FF09C0205C3F4F4F4F5F4F04C066
:10442000215C3F4F4F4F5F4FE0E0F0E02030A0E0D5
:104430003A07A0E04A07A0E45A0710F0E1E0F0E0F4
:1044400079018A0127C06038710564F5FB01E158E4
:10445000FF4FD801C7018F779070A070B070803483
:104460009105A105B10539F4E7FE0DC080E490E0A7
:10447000A0E0B0E004C08FE390E0A0E0B0E0E80E80
:10448000F91E0A1F1B1F17FF05C016950795F79405
:10449000E794319687E016950795F794E7948A9507
:1044A000D1F705C0EE24FF248701EFEFF0E06E2F77
:1044B000679566276795902F9F77D794DD24D794CB
:1044C0008E2F8695492F462B582F5D29B701CA019B
:1044D0001F910F91FF90EF90DF900895FC01DB0199
:1044E000408151812281622F6F7770E0221F222745
:1044F000221F9381892F880F822B282F30E0991F4C
:104500009927991F11969C93119721153105A9F5AB
:10451000411551056105710511F482E037C082E84B
:104520009FEF13969C938E9312979A01AB0167E0CD
:10453000220F331F441F551F6A95D1F783E08C93D8
:104540000DC0220F331F441F551F12968D919C9151
:104550001397019713969C938E931297203080E0C7
:10456000380780E0480780E4580758F314962D93E5
:104570003D934D935C93179708952F3F310579F440
:10458000411551056105710519F484E08C93089576
:1045900064FF03C081E08C9312C01C9210C02F579F
:1045A000304013963C932E93129783E08C9387E0D0
:1045B000440F551F661F771F8A95D1F770641496B4
:1045C0004D935D936D937C93179708951F93DC0132
:1045D000FB019C91923008F447C08081823008F43E
:1045E00043C0943051F411961C91843099F5818127
:1045F000682F70E0611B71093FC0843021F0923058
:1046000031F48230B9F18181882389F12DC011966E
:104610001C9111978230F1F081811817D9F412960C
:104620002D913C911397828193818217930794F087
:1046300028173907BCF014968D919D910D90BC916F
:10464000A02D2481358146815781281739074A07D3
:104650005B0718F4112341F00AC082179307A407DF
:10466000B50740F4112319F061E070E005C06FEF69
:104670007FEF02C060E070E0CB011F910895629F60
:10468000D001739FF001829FE00DF11D649FE00D4A
:10469000F11D929FF00D839FF00D749FF00D659FAB
:1046A000F00D9927729FB00DE11DF91F639FB00DAA
:1046B000E11DF91FBD01CF0111240895AA1BBB1BE9
:1046C00051E107C0AA1FBB1FA617B70710F0A61B12
:1046D000B70B881F991F5A95A9F780959095BC0133
:1046E000CD01089597FB092E07260AD077FD04D047
:1046F000E5DF06D000201AF4709561957F4F08958C
:10470000F6F7909581959F4F0895A1E21A2EAA1B66
:10471000BB1BFD010DC0AA1FBB1FEE1FFF1FA21771
:10472000B307E407F50720F0A21BB30BE40BF50B6E
:10473000661F771F881F991F1A9469F760957095F7
:10474000809590959B01AC01BD01CF01089597FB29
:10475000092E05260ED057FD04D0D7DF0AD0001C45
:1047600038F450954095309521953F4F4F4F5F4F0E
:104770000895F6F790958095709561957F4F8F4FCE
:104780009F4F08952F923F924F925F926F927F9228
:104790008F929F92AF92BF92CF92DF92EF92FF9251
:1047A0000F931F93CF93DF93CDB7DEB7CA1BDB0BFD
:1047B0000FB6F894DEBF0FBECDBF09942A883988A2
:1047C00048885F846E847D848C849B84AA84B984A9
:1047D000C884DF80EE80FD800C811B81AA81B981B5
:1047E000CE0FD11D0FB6F894DEBF0FBECDBFED01C9
:1047F0000895662777270C945D24FC018827992764
:10480000E89421912032E9F3293010F02E30C8F3DA
:104810002B3241F02D3239F4689404C00E942D24CB
:10482000820F911D219120532A30C0F31EF49095E0
:1048300081959F4F0895FB01DC010D900020E9F761
:10484000119701900D920020E1F70895FB01DC0122
:1048500001900D920020E1F708957AE0979F902D46
:10486000879F802D910D11240895DC01CB01FC015F
:10487000F999FECF06C0F2BDE1BDF89A319600B4B9
:104880000D9241505040B8F70895DC01CB0103C0B0
:104890002D910E94502441505040D0F70895262F6A
:1048A000F999FECF1FBA92BD81BD20BD0FB6F89415
:1048B000FA9AF99A0FBE019608958F929F92AF923D
:1048C000BF92CF92DF92EF92FF920F931F93CF93FD
:1048D000DF93EC015B016115710519F0FB01918318
:1048E0008083F9908F2D90E00E94CB25892BC9F70A
:1048F000FDE2FF1621F4F990EE24E39405C02BE2CB
:10490000F21609F4F990EE248E0101501040C8010E
:104910006CEC70E043E050E00E94D325892B01F558
:104920008E010E5F1F4FC8016FEC70E045E050E054
:104930000E94D325892B19F48E01095F1F4FA11402
:10494000B10419F0F50111830083E0FC04C070E0AC
:1049500090E080E814C070E090E080E86FEF08C15C
:10496000C80164ED70E043E050E00E94D325892B3C
:1049700069F4A114B10429F470E090E080EC6FE7D1
:10498000F7C02296F501D183C083F6CF88249924FD
:1049900040E050E060E070E0EF2DE053EA30A0F539
:1049A000F2E0EF2A8E2D90E09C0128703070E2FE3C
:1049B00006C0232B79F50894811C911C2BC0232B56
:1049C00019F0089481089108DB01CA0112E0880FF0
:1049D000991FAA1FBB1F1A95D1F7480F591F6A1FAD
:1049E0007B1F440F551F661F771F4E0F511D611D02
:1049F000711D483929E9520729E9620729E172073F
:104A000048F084E0E82A06C0EE3F31F4E3FC39C008
:104A100098E0E92AF990C0CFE53311F0E53189F546
:104A200029912D3219F4E0E1EE2A05C02B3219F05C
:104A300081E090E003C0299182E090E0E22FE05312
:104A4000EA3018F0C81BD90B1CC020E030E0FCE0B5
:104A500020383F075CF4C901880F991F880F991F00
:104A6000280F391F220F331F2E0F311DE991E053FC
:104A7000EA3068F3E4FE03C0309521953F4F820E83
:104A8000931ECE2CDD24E1FE07C0A114B10421F059
:104A90002197F501D183C083CB01BA010E94EF2594
:104AA0007B018C01F3E0CF22DD2423E0C216D10488
:104AB00021F417FB109517F9109557016801C801EB
:104AC000B70120E030E040E050E00E94EB25882371
:104AD00009F44AC097FE0DC02BEEE22E20E0F22E24
:104AE0009094819491089394C0E2D0E000E010E0AB
:104AF00012C093E0E92E91E0F92EF6CFF70125914F
:104B0000359145915491C601B5010E941B205B016E
:104B10006C018C1A9D0A8C169D0684F7D595C79555
:104B20000F5F1F4F0630110529F08CEF9FEFE80E45
:104B3000F91EF1CFC501D6017C018D018C2D880FA6
:104B40008D2D881F8F3F51F0C601B50120E030E068
:104B500040E050E00E94EB25882331F482E290E0AF
:104B60009093AD108093AC107E2D9F2D802F612FE0
:104B7000272F392F482F562FB901CA01DF91CF9126
:104B80001F910F91FF90EF90DF90CF90BF90AF906B
:104B90009F908F900895911183C0803219F08950B1
:104BA0008550D0F70895FB01DC014150504088F05A
:104BB0008D9181341CF08B350CF4805E65916134ED
:104BC0001CF06B350CF4605E861B611171F3990B60
:104BD0000895881BFCCF40D008F481E00895E89444
:104BE00009C097FB3EF490958095709561957F4F35
:104BF0008F4F9F4F9923A9F0F92F96E9BB279395E3
:104C0000F695879577956795B795F111F8CFFAF4F2
:104C1000BB0F11F460FF1BC06F5F7F4F8F4F9F4F23
:104C200016C0882311F096E911C0772321F09EE881
:104C3000872F762F05C0662371F096E8862F70E0E7
:104C400060E02AF09A95660F771F881FDAF7880FC1
:104C50009695879597F90895990F0008550FAA0B17
:104C6000E0E8FEEF16161706E807F907C0F012167F
:104C70001306E407F50798F0621B730B840B950B82
:104C800039F40A2661F0232B242B252B21F40895D7
:104C90000A2609F4A140A6958FEF811D811D089574
:0A4CA000992788270895F894FFCFA4
:104CAA00526561645F53657475703A20000A0D009D
:104CBA0057726F6E672045454D414749433A200078
:104CCA002F00B400000000000000000000000000F7
:104CDA0000000000000000000000000000000000CA
:104CEA000000000064006400640064006400640062
:104CFA006400640009120D0810040B0E0214070167
:104D0A000F050C0009120D0810040B0E02140701FE
:104D1A000F050C000A0A0A0A0A0A0A0A0A0A0A0AF1
:104D2A000A0A0A0A14141414141414141414141461
:104D3A00141414141E1E1E1E1E1E1E1E1E1E1E1EB1
:104D4A001E1E1E1E64646464646464646464646431
:104D5A0064646464000102030405060708090A0B77
:104D6A000C0D0E0F0E0F14150C100B191A1116122A
:104D7A000D171318110C1A150F10130B0E180D1608
:104D8A001719121414120D0F181316110C1A100BEE
:104D9A000E15191716130E140F181510190B0C1AD5
:104DAA00120D171115101317120E0C1A0B0F110DE5
:104DBA00161814190E0F14150C100B191A111612B5
:104DCA000D17131819110C1A150B140F1810120EAF
:104DDA00170D13161613180D170F100B190E12159F
:104DEA0014110C1A0E17120F110C1A1510160B1497
:104DFA0019130D180B0C0D0E0F1011121314151692
:104E0A001718191A6009455252310D0A00455252B3
:104E1A00320D0A00455252330D0A00455252340DE2
:104E2A000A0054454D323A20002E000A0D00505215
:104E3A0045323A200043414C493A20003B000305E1
:104E4A00080E1A302E382D31333130303630393899
:104E5A0034000A0D535953494E464F3A7A696762EC
:104E6A0069742F72782D70706D2F61746D656C2F57
:104E7A00302E382D313331303036303938340A0D4E
:104E8A000053434E003B00200A0D52534900200AAA
:104E9A000D4C514900200A0D41444300200A0D439C
:104EAA00485600200A0D46535600200A0D45544321
:104EBA003B00200A0D47505300200A0D002D2D2DCE
:104ECA002D2D2D2D2D2D2D2D2D2D2D2D2D2D2D2D08
:104EDA002D2D2D2D2052434F50454E3234202D2D4D
:104EEA002D2D2D2D2D2D2D2D2D2D2D2D2D2D2D2DE8
:104EFA002D2D2D2D2D0A0D00496E666F3A2020208A
:104F0A002020202020205A69676269742052582084
:104F1A00384368616E6E656C2D50504D204F757424
:104F2A007075740A0D0053797374656D3A202020E8
:104F3A00202020207A69676269742F72782D707038
:104F4A006D2F61746D656C2F302E382D31333130F1
:104F5A003036303938340A0D004472697665723A4F
:104F6A00202020202020200070706D2D6F75742065
:104F7A00006E617574696328004368616E6E656CC2
:104F8A00732D3E536572766F2D003B2000780075B5
:104F9A007329200074656C656D65747269652000FB
:104FAA002020202020202020202020202020200A0D
:104FBA000D0050726F746F636F6C202020202020C8
:104FCA0000647373732000666873732000746873D7
:104FDA007320006C697374656E2D6265666F726505
:104FEA002D74616C6B2000525353492864426D2919
:104FFA003A20202020002C002020202020202020C1
:10500A00202020202020200A0D4E4F495345286495
:10501A00426D293A20202000202020202020202014
:10502A00202020202020200A0D534E2D4469666638
:10503A00286442293A2020002020202020202020F5
:10504A00202020202020200A0D4C51493A202020DF
:10505A002020202020202000202020202020202066
:10506A00202020202020200A0D4552524F52533A28
:10507A00202020202020200028002F002000252981
:10508A002020202020202020202020202020200A2C
:10509A000D484F50503A2020202020202020200068
:1050AA0020202020202020202020202020202020F6
:1050BA00200A0D547849443A20202020202020201C
:1050CA002000202800292020202020202020202005
:1050DA0020202020200A0D5345513A20202020204C
:1050EA0020202020200020202020202020202020D6
:1050FA0020200A0D0041444327733A202020202013
:10510A00202020303D0020313D0020323D00203358
:10511A003D00202020200A0D004F534343414C20DC
:10512A002020202020202000202020202020200AAB
:10513A000D005461626C65733A20202020202020E3
:10514A00002C200056616C756573202020202020D9
:10515A002020004C6173742D4D756C74694E756D09
:10516A0020004D756C746976616C7565732020201A
:10517A00002D3E00292000202020202020200A0D7A
:10518A004D756C746976616C756573322020004DBB
:10519A00543A003A0020200A0D002D2D2D2D2D2DD8
:1051AA002D2D2D2D2D2D2D2D2D2D2D2D2D2D2D0A48
:1051BA000D003E003D004D453A000A0D0072636F36
:1051CA0070656E32342D727820285A696762697464
:1051DA0020525820384368616E6E656C2D50504DD0
:1051EA00204F7574707574290A0D005365747469BB
:1051FA006E672046616C65736176652D56616C75C4
:10520A0065730A0D0053657475702D536176656474
:10521A000A0D004D756C746970726F702D53657448
:10522A0074696E67730A0D002E2E2E73617665649B
:10523A002E2E2E002E2E2E72657365742E2E2E00A3
:10524A0062696E642E2E2E2E0A0D000103030303DB
:10525A00000000000000000003030303030303032C
:10526A0004040404040404040404040404040404F4
:10527A0004040404040404040202030202030303F0
:10528A00030203030303020303030303380E3C0E62
:10529A003D0E3E0E3F0E400E420E440E460E480E86
:1052AA004A0E4C0E4E0E500E510E520E530E540E06
:1052BA00550E560E570E580E590E5A0E5B0E5C0EB0
:1052CA005D0E5E0E5F0E600E610E620E630E640E60
:1052DA00650E660E670E680E690E6A0E6B0E6C0E10
:1052EA006D0E6E0E6F0E700E720E740E750E770EB8
:1052FA00790E7A0E7B0E7C0E7D0E7F0E800E810E4D
:10530A00820E830E850E860E870E880E890E6964BC
:10531A00007461626C650074696D657461626C65C4
:10532A00004661696C736176654D6F64650046611C
:10533A00696C73617665536574004661696C736163
:10534A00766556616C7565735F31004661696C7389
:10535A0061766556616C7565735F32004661696C8A
:10536A007361766556616C7565735F330046616972
:10537A006C7361766556616C7565735F340046615E
:10538A00696C7361766556616C7565735F35004645
:10539A0061696C7361766556616C7565735F360019
:1053AA004661696C7361766556616C7565735F37C2
:1053BA00004661696C7361766556616C7565735FE9
:1053CA003800536572766F4D61705F3100536572B4
:1053DA00766F4D61705F3200536572766F4D617002
:1053EA005F3300536572766F4D61705F34005365A9
:1053FA0072766F4D61705F3500536572766F4D61DD
:10540A00705F3600536572766F4D61705F37005377
:10541A006572766F4D61705F3800536572766F44BE
:10542A0075616C526174655F3100536572766F44C1
:10543A0075616C526174655F3200536572766F44B0
:10544A0075616C526174655F3300536572766F449F
:10545A0075616C526174655F3400536572766F448E
:10546A0075616C526174655F3500536572766F447D
:10547A0075616C526174655F3600536572766F446C
:10548A0075616C526174655F3700536572766F445B
:10549A0075616C526174655F3800536572766F414D
:1054AA00747655705F3100536572766F4174765524
:1054BA00705F3200536572766F41747655705F3350
:1054CA0000536572766F41747655705F3400536588
:1054DA0072766F41747655705F3500536572766FD8
:1054EA0041747655705F3600536572766F417476F3
:1054FA0055705F3700536572766F41747655705FE9
:10550A003800536572766F417476446F776E5F31F7
:10551A0000536572766F417476446F776E5F32001E
:10552A00536572766F417476446F776E5F330053BA
:10553A006572766F417476446F776E5F3400536597
:10554A0072766F417476446F776E5F350053657279
:10555A00766F417476446F776E5F36005365727664
:10556A006F417476446F776E5F3700536572766F5A
:10557A00417476446F776E5F380050574D526174AC
:10558A00655F310050574D526174655F320050506B
:10559A004D4368616E6E656C730050504D53796E61
:1055AA00630050504D53686966740050504D496EFF
:1055BA0076657274006D756C74695F6368616E6E8E
:1055CA00656C006D756C74695F6368616E6E656C9D
:1055DA0073006D756C74695F6D73796E635F6E7558
:1055EA006D006D756C74695F6D73796E635F6C6560
:1055FA006E006D756C74695F6368616E6E656C6D63
:10560A006170006D756C7469325F6368616E6E6596
:10561A006C006D756C7469325F6368616E6E656C7F
:10562A0073006D756C7469325F6D73796E635F6E4A
:10563A00756D006D756C7469325F6D73796E635F39
:10564A006C656E006D756C7469325F6368616E6E4D
:10565A00656C6D6170006D656E755F6C656E00637B
:10566A0073765F6F75747075740073617665006D1B
:10567A00756C7469736574006E087108770881081F
:10568A008E089A08AB08BC08CD08DE08EF080009A6
:10569A00110922092D09380943094E0959096409D2
:1056AA006F097A098A099A09AA09BA09CA09DA0993
:1056BA00EA09FA09070A140A210A2E0A3B0A480AC1
:1056CA00550A620A710A800A8F0A9E0AAD0ABC0A42
:1056DA00CB0ADA0AE40AEE0AFA0A020B0B0B150BDA
:1056EA00230B320B420B520B630B720B820B930B85
:1056FA00A40BB60BBF0BCA0BCF0B476C6F62616C66
:10570A00004661696C7361766500536572766F2D28
:10571A004D6170004475616C726174650041747604
:10572A002D5570004174762D446F776E0050574D99
:10573A002D4F75747075740050504D2D4F757470DF
:10574A007574004D756C746970726F70004D756C6C
:10575A00746970726F7032004D656E75005A0C6113
:10576A000C6A0C740C7D0C840C8D0C980CA30CAD7B
:10577A000CB80C00030D151D252D2F33383D030AD7
:10578A0008080808020405050401010101010101D4
:10579A0001010101010101010101010101010101EF
:1057AA00010101010101010101FF010000000000E6
:0457BA0000000000EB
:00000001FF
